 popframe003

 Timestamp is 2ebf369b (reproducible build file hash)

 Preferred load address is 0000000180000000

 Start         Length     Name                   Class
 0001:00000000 00002d80H .text$mn                CODE
 0001:00002d80 00000036H .text$mn$00             CODE
 0001:00002db6 00000092H .text$x                 CODE
 0002:00000000 00000190H .idata$5                DATA
 0002:00000190 00000038H .00cfg                  DATA
 0002:000001c8 00000008H .CRT$XCA                DATA
 0002:000001d0 00000008H .CRT$XCZ                DATA
 0002:000001d8 00000008H .CRT$XIA                DATA
 0002:000001e0 00000008H .CRT$XIC                DATA
 0002:000001e8 00000008H .CRT$XIZ                DATA
 0002:000001f0 00000008H .CRT$XLA                DATA
 0002:000001f8 00000008H .CRT$XLZ                DATA
 0002:00000200 00000008H .CRT$XPA                DATA
 0002:00000208 00000008H .CRT$XPZ                DATA
 0002:00000210 00000008H .CRT$XTA                DATA
 0002:00000218 00000008H .CRT$XTZ                DATA
 0002:00000220 00000000H .gehcont$y              DATA
 0002:00000220 00000000H .gfids$y                DATA
 0002:00000220 00001ee0H .rdata                  DATA
 0002:00002100 00000000H .rdata$CastGuardVftablesA DATA
 0002:00002100 00000000H .rdata$CastGuardVftablesC DATA
 0002:00002100 00000028H .rdata$T                DATA
 0002:00002128 000000b0H .rdata$voltmd           DATA
 0002:000021d8 00000318H .rdata$zzzdbg           DATA
 0002:000024f0 00000008H .rtc$IAA                DATA
 0002:000024f8 00000008H .rtc$IZZ                DATA
 0002:00002500 00000008H .rtc$TAA                DATA
 0002:00002508 00000008H .rtc$TZZ                DATA
 0002:00002510 00000004H .tls                    DATA
 0002:00002514 00000004H .tls$                   DATA
 0002:00002518 00000008H .tls$ZZZ                DATA
 0002:00002520 000002d0H .xdata                  DATA
 0002:000027f0 00000410H .edata                  DATA
 0002:00002c00 00000064H .idata$2                DATA
 0002:00002c64 00000014H .idata$3                DATA
 0002:00002c78 00000190H .idata$4                DATA
 0002:00002e08 00000414H .idata$6                DATA
 0003:00000000 00000080H .data                   DATA
 0003:00000080 0001b388H .bss                    DATA
 0004:00000000 0000039cH .pdata                  DATA

  Address         Publics by Value              Rva+Base               Lib:Object

 0000:00000000       __AbsoluteZero             0000000000000000     <absolute>
 0000:00000000       ___safe_se_handler_count   0000000000000000     <absolute>
 0000:00000000       ___safe_se_handler_table   0000000000000000     <absolute>
 0000:00000000       __arm64x_extra_rfe_table   0000000000000000     <absolute>
 0000:00000000       __arm64x_extra_rfe_table_size 0000000000000000     <absolute>
 0000:00000000       __arm64x_native_entrypoint 0000000000000000     <absolute>
 0000:00000000       __arm64x_redirection_metadata 0000000000000000     <absolute>
 0000:00000000       __arm64x_redirection_metadata_count 0000000000000000     <absolute>
 0000:00000000       __dynamic_value_reloc_table 0000000000000000     <absolute>
 0000:00000000       __enclave_config           0000000000000000     <absolute>
 0000:00000000       __guard_check_icall_a64n_fptr 0000000000000000     <absolute>
 0000:00000000       __guard_eh_cont_count      0000000000000000     <absolute>
 0000:00000000       __guard_eh_cont_table      0000000000000000     <absolute>
 0000:00000000       __guard_fids_count         0000000000000000     <absolute>
 0000:00000000       __guard_fids_table         0000000000000000     <absolute>
 0000:00000000       __guard_iat_count          0000000000000000     <absolute>
 0000:00000000       __guard_iat_table          0000000000000000     <absolute>
 0000:00000000       __guard_longjmp_count      0000000000000000     <absolute>
 0000:00000000       __guard_longjmp_table      0000000000000000     <absolute>
 0000:00000000       __hybrid_auxiliary_iat     0000000000000000     <absolute>
 0000:00000000       __hybrid_auxiliary_iat_copy 0000000000000000     <absolute>
 0000:00000000       __hybrid_code_map          0000000000000000     <absolute>
 0000:00000000       __hybrid_code_map_count    0000000000000000     <absolute>
 0000:00000000       __x64_code_ranges_to_entry_points 0000000000000000     <absolute>
 0000:00000000       __x64_code_ranges_to_entry_points_count 0000000000000000     <absolute>
 0000:00000100       __guard_flags              0000000000000100     <absolute>
 0000:00000000       __ImageBase                0000000180000000     <linker-defined>
 0001:00000000       ?NewObject@JNIEnv_@@QEAAPEAV_jobject@@PEAV_jclass@@PEAU_jmethodID@@ZZ 0000000180001000 f i libpopframe003.obj
 0001:00000024       ?SetEventNotificationMode@_jvmtiEnv@@QEAA?AW4jvmtiError@@W4jvmtiEventMode@@W4jvmtiEvent@@PEAV_jobject@@ZZ 0000000180001024 f i libpopframe003.obj
 0001:0000002c       ?TranslateError@@YAPEBDW4jvmtiError@@@Z 000000018000102c f   libpopframe003.obj
 0001:000002e4       ?nsk_jni_check_exception@@YAHPEAUJNIEnv_@@QEBDH@Z 00000001800012e4 f   libpopframe003.obj
 0001:00000428       ?nsk_jni_lverify@@YAHHPEAUJNIEnv_@@HQEBDH1ZZ 0000000180001428 f   libpopframe003.obj
 0001:000004c8       Agent_Initialize           00000001800014c8 f   libpopframe003.obj
 0001:00000670       Agent_OnAttach             0000000180001670 f   libpopframe003.obj
 0001:00000670       Agent_OnLoad               0000000180001670 f   libpopframe003.obj
 0001:00000678       FramePop                   0000000180001678 f   libpopframe003.obj
 0001:000006cc       Java_nsk_jvmti_PopFrame_popframe003_doPopFrame 00000001800016cc f   libpopframe003.obj
 0001:00000888       Java_nsk_jvmti_PopFrame_popframe003_resThread 0000000180001888 f   libpopframe003.obj
 0001:00000900       Java_nsk_jvmti_PopFrame_popframe003_suspThread 0000000180001900 f   libpopframe003.obj
 0001:00000978       Java_nsk_jvmti_unit_FollowReferences_FollowRefObjects_addRefToVerify 0000000180001978 f   libpopframe003.obj
 0001:00000b34       Java_nsk_jvmti_unit_FollowReferences_FollowRefObjects_getTag 0000000180001b34 f   libpopframe003.obj
 0001:00000bf0       Java_nsk_jvmti_unit_FollowReferences_FollowRefObjects_resetRefsToVerify 0000000180001bf0 f   libpopframe003.obj
 0001:00000bf8       Java_nsk_jvmti_unit_FollowReferences_FollowRefObjects_resetTags 0000000180001bf8 f   libpopframe003.obj
 0001:00000c3c       Java_nsk_jvmti_unit_FollowReferences_FollowRefObjects_setTag 0000000180001c3c f   libpopframe003.obj
 0001:00000e88       Java_nsk_share_jvmti_ArgumentHandler_getAgentOptionsString 0000000180001e88 f   libpopframe003.obj
 0001:00000f34       Java_nsk_share_jvmti_DebugeeClass_checkStatus 0000000180001f34 f   libpopframe003.obj
 0001:00000fbc       Java_nsk_share_jvmti_DebugeeClass_resetAgentData 0000000180001fbc f   libpopframe003.obj
 0001:0000101c       Java_nsk_share_jvmti_RedefineAgent_agentStatus 000000018000201c f   libpopframe003.obj
 0001:00001028       Java_nsk_share_jvmti_RedefineAgent_isRedefined 0000000180002028 f   libpopframe003.obj
 0001:00001034       Java_nsk_share_jvmti_RedefineAgent_redefineAttempted 0000000180002034 f   libpopframe003.obj
 0001:00001040       MA_checkStatus             0000000180002040 f   libpopframe003.obj
 0001:000010e4       MethodExit                 00000001800020e4 f   libpopframe003.obj
 0001:00001138       __local_stdio_printf_options 0000000180002138 f i libpopframe003.obj
 0001:00001308       exitOnError                0000000180002308 f   libpopframe003.obj
 0001:000013bc       fprintf                    00000001800023bc f i libpopframe003.obj
 0001:00001400       nsk_jvmti_lverify          0000000180002400 f   libpopframe003.obj
 0001:000014f0       nsk_jvmti_resetAgentData   00000001800024f0 f   libpopframe003.obj
 0001:00001564       nsk_lcomplain              0000000180002564 f   libpopframe003.obj
 0001:00001584       nsk_ldisplay               0000000180002584 f   libpopframe003.obj
 0001:000015a4       nsk_ltrace                 00000001800025a4 f   libpopframe003.obj
 0001:000015c4       nsk_lvcomplain             00000001800025c4 f   libpopframe003.obj
 0001:0000177c       nsk_lvdisplay              000000018000277c f   libpopframe003.obj
 0001:000017c8       nsk_lverify                00000001800027c8 f   libpopframe003.obj
 0001:00001824       nsk_lvtrace                0000000180002824 f   libpopframe003.obj
 0001:00001884       nsk_printf                 0000000180002884 f   libpopframe003.obj
 0001:000018ac       nsk_vprintf                00000001800028ac f   libpopframe003.obj
 0001:00001960       printf                     0000000180002960 f i libpopframe003.obj
 0001:00001e60       __raise_securityfailure    0000000180002e60 f   MSVCRT:gs_report.obj
 0001:00001e94       __report_gsfailure         0000000180002e94 f   MSVCRT:gs_report.obj
 0001:000020d4       __GSHandlerCheck           00000001800030d4 f   MSVCRT:gshandler.obj
 0001:000020f4       __GSHandlerCheckCommon     00000001800030f4 f   MSVCRT:gshandler.obj
 0001:00002160       __security_check_cookie    0000000180003160 f   MSVCRT:amdsecgs.obj
 0001:000024a0       _DllMainCRTStartup         00000001800034a0 f   MSVCRT:dll_dllmain.obj
 0001:000024e0       __scrt_acquire_startup_lock 00000001800034e0 f   MSVCRT:utility.obj
 0001:0000251c       __scrt_dllmain_after_initialize_c 000000018000351c f   MSVCRT:utility.obj
 0001:00002550       __scrt_dllmain_before_initialize_c 0000000180003550 f   MSVCRT:utility.obj
 0001:00002568       __scrt_dllmain_crt_thread_attach 0000000180003568 f   MSVCRT:utility.obj
 0001:00002590       __scrt_dllmain_crt_thread_detach 0000000180003590 f   MSVCRT:utility.obj
 0001:000025a8       __scrt_dllmain_exception_filter 00000001800035a8 f   MSVCRT:utility.obj
 0001:00002608       __scrt_dllmain_uninitialize_c 0000000180003608 f   MSVCRT:utility.obj
 0001:00002638       __scrt_dllmain_uninitialize_critical 0000000180003638 f   MSVCRT:utility.obj
 0001:0000264c       __scrt_initialize_crt      000000018000364c f   MSVCRT:utility.obj
 0001:00002698       __scrt_initialize_onexit_tables 0000000180003698 f   MSVCRT:utility.obj
 0001:00002724       __scrt_is_nonwritable_in_current_image 0000000180003724 f   MSVCRT:utility.obj
 0001:000027bc       __scrt_release_startup_lock 00000001800037bc f   MSVCRT:utility.obj
 0001:000027e0       __scrt_uninitialize_crt    00000001800037e0 f   MSVCRT:utility.obj
 0001:0000280c       _onexit                    000000018000380c f   MSVCRT:utility.obj
 0001:00002848       atexit                     0000000180003848 f   MSVCRT:utility.obj
 0001:00002860       __crt_debugger_hook        0000000180003860 f   MSVCRT:utility_desktop.obj
 0001:00002868       __scrt_fastfail            0000000180003868 f   MSVCRT:utility_desktop.obj
 0001:000029b4       _guard_check_icall_nop     00000001800039b4 f i MSVCRT:guard_support.obj
 0001:000029b8       __security_init_cookie     00000001800039b8 f   MSVCRT:gs_support.obj
 0001:00002a64       DllMain                    0000000180003a64 f   MSVCRT:dll_dllmain_stub.obj
 0001:00002a88       ?__scrt_initialize_type_info@@YAXXZ 0000000180003a88 f   MSVCRT:tncleanup.obj
 0001:00002a98       ?__scrt_uninitialize_type_info@@YAXXZ 0000000180003a98 f   MSVCRT:tncleanup.obj
 0001:00002aa4       __local_stdio_scanf_options 0000000180003aa4 f i MSVCRT:default_local_stdio_options.obj
 0001:00002aac       __scrt_initialize_default_local_stdio_options 0000000180003aac f   MSVCRT:default_local_stdio_options.obj
 0001:00002ac8       __scrt_get_dyn_tls_init_callback 0000000180003ac8 f   MSVCRT:dyn_tls_init.obj
 0001:00002ad0       _RTC_Initialize            0000000180003ad0 f   MSVCRT:initsect.obj
 0001:00002b0c       _RTC_Terminate             0000000180003b0c f   MSVCRT:initsect.obj
 0001:00002b48       __isa_available_init       0000000180003b48 f   MSVCRT:cpu_disp.obj
 0001:00002cf4       _get_startup_argv_mode     0000000180003cf4 f   MSVCRT:argv_mode.obj
 0001:00002cfc       __scrt_is_ucrt_dll_in_use  0000000180003cfc f   MSVCRT:ucrt_detection.obj
 0001:00002d10       memcpy                     0000000180003d10 f   vcruntime:VCRUNTIME140.dll
 0001:00002d16       memset                     0000000180003d16 f   vcruntime:VCRUNTIME140.dll
 0001:00002d1c       strchr                     0000000180003d1c f   vcruntime:VCRUNTIME140.dll
 0001:00002d22       __C_specific_handler       0000000180003d22 f   vcruntime:VCRUNTIME140.dll
 0001:00002d28       __std_type_info_destroy_list 0000000180003d28 f   vcruntime:VCRUNTIME140.dll
 0001:00002d2e       strlen                     0000000180003d2e f   ucrt:api-ms-win-crt-string-l1-1-0.dll
 0001:00002d34       _initterm                  0000000180003d34 f   ucrt:api-ms-win-crt-runtime-l1-1-0.dll
 0001:00002d3a       _initterm_e                0000000180003d3a f   ucrt:api-ms-win-crt-runtime-l1-1-0.dll
 0001:00002d40       _seh_filter_dll            0000000180003d40 f   ucrt:api-ms-win-crt-runtime-l1-1-0.dll
 0001:00002d46       _configure_narrow_argv     0000000180003d46 f   ucrt:api-ms-win-crt-runtime-l1-1-0.dll
 0001:00002d4c       _initialize_narrow_environment 0000000180003d4c f   ucrt:api-ms-win-crt-runtime-l1-1-0.dll
 0001:00002d52       _initialize_onexit_table   0000000180003d52 f   ucrt:api-ms-win-crt-runtime-l1-1-0.dll
 0001:00002d58       _register_onexit_function  0000000180003d58 f   ucrt:api-ms-win-crt-runtime-l1-1-0.dll
 0001:00002d5e       _execute_onexit_table      0000000180003d5e f   ucrt:api-ms-win-crt-runtime-l1-1-0.dll
 0001:00002d64       _crt_atexit                0000000180003d64 f   ucrt:api-ms-win-crt-runtime-l1-1-0.dll
 0001:00002d6a       _cexit                     0000000180003d6a f   ucrt:api-ms-win-crt-runtime-l1-1-0.dll
 0001:00002d70       __acrt_initialize          0000000180003d70 f   MSVCRT:ucrt_stubs.obj
 0001:00002d70       __acrt_thread_attach       0000000180003d70 f   MSVCRT:ucrt_stubs.obj
 0001:00002d70       __acrt_thread_detach       0000000180003d70 f   MSVCRT:ucrt_stubs.obj
 0001:00002d70       __acrt_uninitialize        0000000180003d70 f   MSVCRT:ucrt_stubs.obj
 0001:00002d70       __acrt_uninitialize_critical 0000000180003d70 f   MSVCRT:ucrt_stubs.obj
 0001:00002d70       __scrt_stub_for_acrt_initialize 0000000180003d70 f   MSVCRT:ucrt_stubs.obj
 0001:00002d70       __scrt_stub_for_acrt_thread_attach 0000000180003d70 f   MSVCRT:ucrt_stubs.obj
 0001:00002d70       __scrt_stub_for_acrt_thread_detach 0000000180003d70 f   MSVCRT:ucrt_stubs.obj
 0001:00002d70       __scrt_stub_for_acrt_uninitialize 0000000180003d70 f   MSVCRT:ucrt_stubs.obj
 0001:00002d70       __scrt_stub_for_acrt_uninitialize_critical 0000000180003d70 f   MSVCRT:ucrt_stubs.obj
 0001:00002d70       __vcrt_initialize          0000000180003d70 f   MSVCRT:ucrt_stubs.obj
 0001:00002d70       __vcrt_thread_attach       0000000180003d70 f   MSVCRT:ucrt_stubs.obj
 0001:00002d70       __vcrt_thread_detach       0000000180003d70 f   MSVCRT:ucrt_stubs.obj
 0001:00002d70       __vcrt_uninitialize        0000000180003d70 f   MSVCRT:ucrt_stubs.obj
 0001:00002d70       __vcrt_uninitialize_critical 0000000180003d70 f   MSVCRT:ucrt_stubs.obj
 0001:00002d74       __scrt_stub_for_is_c_termination_complete 0000000180003d74 f   MSVCRT:ucrt_stubs.obj
 0001:00002d74       _is_c_termination_complete 0000000180003d74 f   MSVCRT:ucrt_stubs.obj
 0001:00002d90       _guard_dispatch_icall_nop  0000000180003d90 f   MSVCRT:guard_dispatch.obj
 0001:00002db0       _guard_xfg_dispatch_icall_nop 0000000180003db0 f   MSVCRT:guard_xfg_dispatch.obj
 0002:00000000       __imp_RtlCaptureContext    0000000180004000     kernel32:KERNEL32.dll
 0002:00000008       __imp_RtlLookupFunctionEntry 0000000180004008     kernel32:KERNEL32.dll
 0002:00000010       __imp_RtlVirtualUnwind     0000000180004010     kernel32:KERNEL32.dll
 0002:00000018       __imp_UnhandledExceptionFilter 0000000180004018     kernel32:KERNEL32.dll
 0002:00000020       __imp_SetUnhandledExceptionFilter 0000000180004020     kernel32:KERNEL32.dll
 0002:00000028       __imp_GetCurrentProcess    0000000180004028     kernel32:KERNEL32.dll
 0002:00000030       __imp_TerminateProcess     0000000180004030     kernel32:KERNEL32.dll
 0002:00000038       __imp_IsProcessorFeaturePresent 0000000180004038     kernel32:KERNEL32.dll
 0002:00000040       __imp_CloseHandle          0000000180004040     kernel32:KERNEL32.dll
 0002:00000048       __imp_InitializeCriticalSectionAndSpinCount 0000000180004048     kernel32:KERNEL32.dll
 0002:00000050       __imp_DeleteCriticalSection 0000000180004050     kernel32:KERNEL32.dll
 0002:00000058       __imp_CreateEventW         0000000180004058     kernel32:KERNEL32.dll
 0002:00000060       __imp_GetModuleHandleW     0000000180004060     kernel32:KERNEL32.dll
 0002:00000068       __imp_GetProcAddress       0000000180004068     kernel32:KERNEL32.dll
 0002:00000070       __imp_IsDebuggerPresent    0000000180004070     kernel32:KERNEL32.dll
 0002:00000078       __imp_QueryPerformanceCounter 0000000180004078     kernel32:KERNEL32.dll
 0002:00000080       __imp_GetCurrentProcessId  0000000180004080     kernel32:KERNEL32.dll
 0002:00000088       __imp_GetCurrentThreadId   0000000180004088     kernel32:KERNEL32.dll
 0002:00000090       __imp_GetSystemTimeAsFileTime 0000000180004090     kernel32:KERNEL32.dll
 0002:00000098       __imp_DisableThreadLibraryCalls 0000000180004098     kernel32:KERNEL32.dll
 0002:000000a0       __imp_InitializeSListHead  00000001800040a0     kernel32:KERNEL32.dll
 0002:000000a8       \177KERNEL32_NULL_THUNK_DATA 00000001800040a8     kernel32:KERNEL32.dll
 0002:000000b0       __imp_memcpy               00000001800040b0     vcruntime:VCRUNTIME140.dll
 0002:000000b8       __imp_memset               00000001800040b8     vcruntime:VCRUNTIME140.dll
 0002:000000c0       __imp_strchr               00000001800040c0     vcruntime:VCRUNTIME140.dll
 0002:000000c8       __imp___C_specific_handler 00000001800040c8     vcruntime:VCRUNTIME140.dll
 0002:000000d0       __imp___std_type_info_destroy_list 00000001800040d0     vcruntime:VCRUNTIME140.dll
 0002:000000d8       \177VCRUNTIME140_NULL_THUNK_DATA 00000001800040d8     vcruntime:VCRUNTIME140.dll
 0002:000000e0       __imp__errno               00000001800040e0     ucrt:api-ms-win-crt-runtime-l1-1-0.dll
 0002:000000e8       __imp_exit                 00000001800040e8     ucrt:api-ms-win-crt-runtime-l1-1-0.dll
 0002:000000f0       __imp__cexit               00000001800040f0     ucrt:api-ms-win-crt-runtime-l1-1-0.dll
 0002:000000f8       __imp__crt_atexit          00000001800040f8     ucrt:api-ms-win-crt-runtime-l1-1-0.dll
 0002:00000100       __imp__execute_onexit_table 0000000180004100     ucrt:api-ms-win-crt-runtime-l1-1-0.dll
 0002:00000108       __imp__register_onexit_function 0000000180004108     ucrt:api-ms-win-crt-runtime-l1-1-0.dll
 0002:00000110       __imp__initialize_onexit_table 0000000180004110     ucrt:api-ms-win-crt-runtime-l1-1-0.dll
 0002:00000118       __imp__initialize_narrow_environment 0000000180004118     ucrt:api-ms-win-crt-runtime-l1-1-0.dll
 0002:00000120       __imp__configure_narrow_argv 0000000180004120     ucrt:api-ms-win-crt-runtime-l1-1-0.dll
 0002:00000128       __imp__seh_filter_dll      0000000180004128     ucrt:api-ms-win-crt-runtime-l1-1-0.dll
 0002:00000130       __imp__initterm_e          0000000180004130     ucrt:api-ms-win-crt-runtime-l1-1-0.dll
 0002:00000138       __imp__initterm            0000000180004138     ucrt:api-ms-win-crt-runtime-l1-1-0.dll
 0002:00000140       \177api-ms-win-crt-runtime-l1-1-0_NULL_THUNK_DATA 0000000180004140     ucrt:api-ms-win-crt-runtime-l1-1-0.dll
 0002:00000148       __imp___acrt_iob_func      0000000180004148     ucrt:api-ms-win-crt-stdio-l1-1-0.dll
 0002:00000150       __imp_fflush               0000000180004150     ucrt:api-ms-win-crt-stdio-l1-1-0.dll
 0002:00000158       __imp___stdio_common_vsprintf 0000000180004158     ucrt:api-ms-win-crt-stdio-l1-1-0.dll
 0002:00000160       __imp___stdio_common_vfprintf 0000000180004160     ucrt:api-ms-win-crt-stdio-l1-1-0.dll
 0002:00000168       \177api-ms-win-crt-stdio-l1-1-0_NULL_THUNK_DATA 0000000180004168     ucrt:api-ms-win-crt-stdio-l1-1-0.dll
 0002:00000170       __imp__strdup              0000000180004170     ucrt:api-ms-win-crt-string-l1-1-0.dll
 0002:00000170       __imp_strdup               0000000180004170     ucrt:api-ms-win-crt-string-l1-1-0.dll
 0002:00000178       __imp_strlen               0000000180004178     ucrt:api-ms-win-crt-string-l1-1-0.dll
 0002:00000180       __imp_strncpy              0000000180004180     ucrt:api-ms-win-crt-string-l1-1-0.dll
 0002:00000188       \177api-ms-win-crt-string-l1-1-0_NULL_THUNK_DATA 0000000180004188     ucrt:api-ms-win-crt-string-l1-1-0.dll
 0002:00000190       __guard_check_icall_fptr   0000000180004190     MSVCRT:guard_support.obj
 0002:00000198       __guard_xfg_check_icall_fptr 0000000180004198     MSVCRT:guard_support.obj
 0002:000001a0       __guard_dispatch_icall_fptr 00000001800041a0     MSVCRT:guard_support.obj
 0002:000001a8       __guard_xfg_dispatch_icall_fptr 00000001800041a8     MSVCRT:guard_support.obj
 0002:000001b0       __guard_xfg_table_dispatch_icall_fptr 00000001800041b0     MSVCRT:guard_support.obj
 0002:000001b8       __castguard_check_failure_os_handled_fptr 00000001800041b8     MSVCRT:guard_support.obj
 0002:000001c0       __guard_memcpy_fptr        00000001800041c0     vcruntime:softmemtag.obj
 0002:000001c8       __xc_a                     00000001800041c8     MSVCRT:initializers.obj
 0002:000001d0       __xc_z                     00000001800041d0     MSVCRT:initializers.obj
 0002:000001d8       __xi_a                     00000001800041d8     MSVCRT:initializers.obj
 0002:000001e8       __xi_z                     00000001800041e8     MSVCRT:initializers.obj
 0002:000001f0       __xl_a                     00000001800041f0     MSVCRT:tlssup.obj
 0002:000001f8       __xl_z                     00000001800041f8     MSVCRT:tlssup.obj
 0002:00000200       __xp_a                     0000000180004200     MSVCRT:initializers.obj
 0002:00000208       __xp_z                     0000000180004208     MSVCRT:initializers.obj
 0002:00000210       __xt_a                     0000000180004210     MSVCRT:initializers.obj
 0002:00000218       __xt_z                     0000000180004218     MSVCRT:initializers.obj
 0002:00000220       g_refKindStr               0000000180004220     libpopframe003.obj
 0002:000003d0       ??_C@_09BPLDFGCI@unknown_0@ 00000001800043d0     libpopframe003.obj
 0002:000003e0       ??_C@_0BL@FPNMECJD@JVMTI_HEAP_REFERENCE_CLASS@ 00000001800043e0     libpopframe003.obj
 0002:00000400       ??_C@_0BL@FKGKKLNM@JVMTI_HEAP_REFERENCE_FIELD@ 0000000180004400     libpopframe003.obj
 0002:00000420       ??_C@_0CD@CAEHCFJF@JVMTI_HEAP_REFERENCE_ARRAY_ELEM@ 0000000180004420     libpopframe003.obj
 0002:00000448       ??_C@_0CC@DNEBMCNK@JVMTI_HEAP_REFERENCE_CLASS_LOAD@ 0000000180004448     libpopframe003.obj
 0002:00000470       ??_C@_0BN@CJMIPEBB@JVMTI_HEAP_REFERENCE_SIGNERS@ 0000000180004470     libpopframe003.obj
 0002:00000490       ??_C@_0CH@HBOIDPEB@JVMTI_HEAP_REFERENCE_PROTECTION@ 0000000180004490     libpopframe003.obj
 0002:000004b8       ??_C@_0BP@MDKGDGKL@JVMTI_HEAP_REFERENCE_INTERFACE@ 00000001800044b8     libpopframe003.obj
 0002:000004d8       ??_C@_0CC@JJMIHNJH@JVMTI_HEAP_REFERENCE_STATIC_FIE@ 00000001800044d8     libpopframe003.obj
 0002:00000500       ??_C@_0CD@IDHEEGID@JVMTI_HEAP_REFERENCE_CONSTANT_P@ 0000000180004500     libpopframe003.obj
 0002:00000528       ??_C@_0CA@EFFCHNG@JVMTI_HEAP_REFERENCE_SUPERCLASS@ 0000000180004528     libpopframe003.obj
 0002:00000548       ??_C@_0L@PCDFHGCJ@unknown_11@ 0000000180004548     libpopframe003.obj
 0002:00000558       ??_C@_0L@NJBICFOK@unknown_12@ 0000000180004558     libpopframe003.obj
 0002:00000568       ??_C@_0L@MAADBEKL@unknown_13@ 0000000180004568     libpopframe003.obj
 0002:00000578       ??_C@_0L@IPECICGM@unknown_14@ 0000000180004578     libpopframe003.obj
 0002:00000588       ??_C@_0L@JGFJLDCN@unknown_15@ 0000000180004588     libpopframe003.obj
 0002:00000598       ??_C@_0L@LNHEOAOO@unknown_16@ 0000000180004598     libpopframe003.obj
 0002:000005a8       ??_C@_0L@KEGPNBKP@unknown_17@ 00000001800045a8     libpopframe003.obj
 0002:000005b8       ??_C@_0L@CDPHMNGA@unknown_18@ 00000001800045b8     libpopframe003.obj
 0002:000005c8       ??_C@_0L@DKOMPMCB@unknown_19@ 00000001800045c8     libpopframe003.obj
 0002:000005d8       ??_C@_0L@OJGIPJDB@unknown_20@ 00000001800045d8     libpopframe003.obj
 0002:000005e8       ??_C@_0CA@KAOFNDEM@JVMTI_HEAP_REFERENCE_JNI_GLOBAL@ 00000001800045e8     libpopframe003.obj
 0002:00000608       ??_C@_0CC@HPFAJBK@JVMTI_HEAP_REFERENCE_SYSTEM_CLA@ 0000000180004608     libpopframe003.obj
 0002:00000630       ??_C@_0BN@FDEGFOHC@JVMTI_HEAP_REFERENCE_MONITOR@ 0000000180004630     libpopframe003.obj
 0002:00000650       ??_C@_0CB@HKIBCMAJ@JVMTI_HEAP_REFERENCE_STACK_LOCA@ 0000000180004650     libpopframe003.obj
 0002:00000678       ??_C@_0BP@EAACMMOE@JVMTI_HEAP_REFERENCE_JNI_LOCAL@ 0000000180004678     libpopframe003.obj
 0002:00000698       ??_C@_0BM@IJDEOGOE@JVMTI_HEAP_REFERENCE_THREAD@ 0000000180004698     libpopframe003.obj
 0002:000006b8       ??_C@_0BL@EDGPPKC@JVMTI_HEAP_REFERENCE_OTHER@ 00000001800046b8     libpopframe003.obj
 0002:000006d4       ??_C@_04BCJPDBDA@Code@     00000001800046d4     libpopframe003.obj
 0002:000006e0       ??_C@_0BA@OCLMCFKC@LineNumberTable@ 00000001800046e0     libpopframe003.obj
 0002:000006f0       ??_C@_0BD@CPAEPILC@LocalVariableTable@ 00000001800046f0     libpopframe003.obj
 0002:00000708       ??_C@_0BH@NMBDNHBD@LocalVariableTypeTable@ 0000000180004708     libpopframe003.obj
 0002:00000720       ??_C@_0O@HIHEEDNJ@StackMapTable@ 0000000180004720     libpopframe003.obj
 0002:00000730       ??_C@_0L@HCDIAMJG@?9?5?$CFs?0?5?$CFd?3?5@ 0000000180004730     libpopframe003.obj
 0002:00000740       ??_C@_0JI@HLPECLFI@?$CD?5?4?4?4?6?$CD?5ERROR?3?5too?5many?5complai@ 0000000180004740     libpopframe003.obj
 0002:000007e0       ??_C@_0ED@JNEKCCOB@The?5following?5fake?5exception?5st@ 00000001800047e0     libpopframe003.obj
 0002:00000828       ??_C@_0CN@FCNMDFBH@nsk?4share?4Fake_Exception_for_RU@ 0000000180004828     libpopframe003.obj
 0002:00000858       ??_C@_08PGFFNAEI@?$CI?$CFs?3?$CFd?$CJ?5@ 0000000180004858     libpopframe003.obj
 0002:00000868       ??_C@_0DP@IENMAEGI@s?2test?2hotspot?2jtreg?2vmTestbase@ 0000000180004868     libpopframe003.obj
 0002:000008a8       ??_C@_0BL@NDJLFFJB@?7at?5nsk_lvcomplain?$CI?$CFs?3?$CFd?$CJ?6@ 00000001800048a8     libpopframe003.obj
 0002:000008c8       ??_C@_0BC@JOOKAFKF@?$CD?5ERROR?3?5?$CFs?0?5?$CFd?3?5@ 00000001800048c8     libpopframe003.obj
 0002:000008e0       ??_C@_09KJEAHMEH@?$CD?5ERROR?3?5@ 00000001800048e0     libpopframe003.obj
 0002:000008ec       ??_C@_02GPIOPFAK@?$DO?$DO@ 00000001800048ec     libpopframe003.obj
 0002:000008f0       ??_C@_02FODMEDOG@?$DM?$DM@ 00000001800048f0     libpopframe003.obj
 0002:000008f4       ??_C@_02DJGKEECL@?4?4@     00000001800048f4     libpopframe003.obj
 0002:000008f8       ??_C@_0O@CJPGJOAF@?9?5?$CFs?0?5?$CFd?3?5?$CFs?5@ 00000001800048f8     libpopframe003.obj
 0002:00000908       ??_C@_0CB@IAKPDOIC@?$CD?5?5?5verified?5assertion?5is?5FALSE@ 0000000180004908     libpopframe003.obj
 0002:00000930       ??_C@_0CO@LGONDEPD@stdout?3?5fflush?5failed?5?9?5err?$DN?$CFd?5@ 0000000180004930     libpopframe003.obj
 0002:00000960       ??_C@_0CO@KBGKJPBD@stderr?3?5fflush?5failed?5?9?5err?$DN?$CFd?5@ 0000000180004960     libpopframe003.obj
 0002:00000990       ??_C@_0BB@JCNMKLLK@JVMTI_ERROR_NONE@ 0000000180004990     libpopframe003.obj
 0002:000009a8       ??_C@_0BL@LDIMKLPH@JVMTI_ERROR_INVALID_THREAD@ 00000001800049a8     libpopframe003.obj
 0002:000009c8       ??_C@_0CB@PJFPAIKJ@JVMTI_ERROR_INVALID_THREAD_GROU@ 00000001800049c8     libpopframe003.obj
 0002:000009f0       ??_C@_0BN@LLMKHMNF@JVMTI_ERROR_INVALID_PRIORITY@ 00000001800049f0     libpopframe003.obj
 0002:00000a10       ??_C@_0CB@MBOFKAGB@JVMTI_ERROR_THREAD_NOT_SUSPENDE@ 0000000180004a10     libpopframe003.obj
 0002:00000a38       ??_C@_0BN@FABOLPBI@JVMTI_ERROR_THREAD_SUSPENDED@ 0000000180004a38     libpopframe003.obj
 0002:00000a58       ??_C@_0BN@FDGNOBJM@JVMTI_ERROR_THREAD_NOT_ALIVE@ 0000000180004a58     libpopframe003.obj
 0002:00000a78       ??_C@_0BL@GOBIFKNJ@JVMTI_ERROR_INVALID_OBJECT@ 0000000180004a78     libpopframe003.obj
 0002:00000a98       ??_C@_0BK@FCMAJPPC@JVMTI_ERROR_INVALID_CLASS@ 0000000180004a98     libpopframe003.obj
 0002:00000ab8       ??_C@_0BP@IKLLBKEB@JVMTI_ERROR_CLASS_NOT_PREPARED@ 0000000180004ab8     libpopframe003.obj
 0002:00000ad8       ??_C@_0BN@KLPPLKG@JVMTI_ERROR_INVALID_METHODID@ 0000000180004ad8     libpopframe003.obj
 0002:00000af8       ??_C@_0BN@BCEKOKND@JVMTI_ERROR_INVALID_LOCATION@ 0000000180004af8     libpopframe003.obj
 0002:00000b18       ??_C@_0BM@DFDGPME@JVMTI_ERROR_INVALID_FIELDID@ 0000000180004b18     libpopframe003.obj
 0002:00000b38       ??_C@_0BL@NELIEPEC@JVMTI_ERROR_NO_MORE_FRAMES@ 0000000180004b38     libpopframe003.obj
 0002:00000b58       ??_C@_0BJ@BDBECFDM@JVMTI_ERROR_OPAQUE_FRAME@ 0000000180004b58     libpopframe003.obj
 0002:00000b78       ??_C@_0BK@MIIFNLOB@JVMTI_ERROR_TYPE_MISMATCH@ 0000000180004b78     libpopframe003.obj
 0002:00000b98       ??_C@_0BJ@HPCAOILC@JVMTI_ERROR_INVALID_SLOT@ 0000000180004b98     libpopframe003.obj
 0002:00000bb8       ??_C@_0BG@CHILOPNI@JVMTI_ERROR_DUPLICATE@ 0000000180004bb8     libpopframe003.obj
 0002:00000bd0       ??_C@_0BG@DIEMLHKM@JVMTI_ERROR_NOT_FOUND@ 0000000180004bd0     libpopframe003.obj
 0002:00000be8       ??_C@_0BM@NHMCKHOB@JVMTI_ERROR_INVALID_MONITOR@ 0000000180004be8     libpopframe003.obj
 0002:00000c08       ??_C@_0BO@PPEDAJGL@JVMTI_ERROR_NOT_MONITOR_OWNER@ 0000000180004c08     libpopframe003.obj
 0002:00000c28       ??_C@_0BG@FCAIPEID@JVMTI_ERROR_INTERRUPT@ 0000000180004c28     libpopframe003.obj
 0002:00000c40       ??_C@_0CB@EGDBNKOI@JVMTI_ERROR_INVALID_CLASS_FORMA@ 0000000180004c40     libpopframe003.obj
 0002:00000c68       ??_C@_0CG@DGKOGIAL@JVMTI_ERROR_CIRCULAR_CLASS_DEFI@ 0000000180004c68     libpopframe003.obj
 0002:00000c90       ??_C@_0BP@ICEALPKC@JVMTI_ERROR_FAILS_VERIFICATION@ 0000000180004c90     libpopframe003.obj
 0002:00000cb0       ??_C@_0DC@JDACLMIO@JVMTI_ERROR_UNSUPPORTED_REDEFIN@ 0000000180004cb0     libpopframe003.obj
 0002:00000ce8       ??_C@_0DE@GKDKNOMJ@JVMTI_ERROR_UNSUPPORTED_REDEFIN@ 0000000180004ce8     libpopframe003.obj
 0002:00000d20       ??_C@_0BO@LAFKIOG@JVMTI_ERROR_INVALID_TYPESTATE@ 0000000180004d20     libpopframe003.obj
 0002:00000d40       ??_C@_0DH@INDGCLLB@JVMTI_ERROR_UNSUPPORTED_REDEFIN@ 0000000180004d40     libpopframe003.obj
 0002:00000d78       ??_C@_0DE@NHEOMMGI@JVMTI_ERROR_UNSUPPORTED_REDEFIN@ 0000000180004d78     libpopframe003.obj
 0002:00000db0       ??_C@_0CA@EKPNJOEP@JVMTI_ERROR_UNSUPPORTED_VERSION@ 0000000180004db0     libpopframe003.obj
 0002:00000dd0       ??_C@_0BN@OFFMAHHL@JVMTI_ERROR_NAMES_DONT_MATCH@ 0000000180004dd0     libpopframe003.obj
 0002:00000df0       ??_C@_0DN@HHBBLAKE@JVMTI_ERROR_UNSUPPORTED_REDEFIN@ 0000000180004df0     libpopframe003.obj
 0002:00000e30       ??_C@_0DO@HMBGBGNA@JVMTI_ERROR_UNSUPPORTED_REDEFIN@ 0000000180004e30     libpopframe003.obj
 0002:00000e70       ??_C@_0BP@PBECGKHJ@JVMTI_ERROR_UNMODIFIABLE_CLASS@ 0000000180004e70     libpopframe003.obj
 0002:00000e90       ??_C@_0BK@CANILEHF@JVMTI_ERROR_NOT_AVAILABLE@ 0000000180004e90     libpopframe003.obj
 0002:00000eb0       ??_C@_0CE@INJKMEFK@JVMTI_ERROR_MUST_POSSESS_CAPABI@ 0000000180004eb0     libpopframe003.obj
 0002:00000ed8       ??_C@_0BJ@LBFPFPDM@JVMTI_ERROR_NULL_POINTER@ 0000000180004ed8     libpopframe003.obj
 0002:00000ef8       ??_C@_0BP@CHJPNNEM@JVMTI_ERROR_ABSENT_INFORMATION@ 0000000180004ef8     libpopframe003.obj
 0002:00000f18       ??_C@_0BP@OMFMNLC@JVMTI_ERROR_INVALID_EVENT_TYPE@ 0000000180004f18     libpopframe003.obj
 0002:00000f38       ??_C@_0BN@BIBNPHHO@JVMTI_ERROR_ILLEGAL_ARGUMENT@ 0000000180004f38     libpopframe003.obj
 0002:00000f58       ??_C@_0BK@KKNDHDCE@JVMTI_ERROR_NATIVE_METHOD@ 0000000180004f58     libpopframe003.obj
 0002:00000f78       ??_C@_0BK@PMKCFHAE@JVMTI_ERROR_OUT_OF_MEMORY@ 0000000180004f78     libpopframe003.obj
 0002:00000f98       ??_C@_0BK@NNJBDMNB@JVMTI_ERROR_ACCESS_DENIED@ 0000000180004f98     libpopframe003.obj
 0002:00000fb8       ??_C@_0BI@GHECLMNC@JVMTI_ERROR_WRONG_PHASE@ 0000000180004fb8     libpopframe003.obj
 0002:00000fd0       ??_C@_0BF@OLIHJOII@JVMTI_ERROR_INTERNAL@ 0000000180004fd0     libpopframe003.obj
 0002:00000fe8       ??_C@_0BO@EOHGKJHI@JVMTI_ERROR_UNATTACHED_THREAD@ 0000000180004fe8     libpopframe003.obj
 0002:00001008       ??_C@_0CA@LKHFDACL@JVMTI_ERROR_INVALID_ENVIRONMENT@ 0000000180005008     libpopframe003.obj
 0002:00001028       ??_C@_0BA@MMFHLOKK@?$DMunknown?5error?$DO@ 0000000180005028     libpopframe003.obj
 0002:00001038       ??_C@_0CF@CBHOKDB@throwable?5?$DN?5jni?9?$DOExceptionOccur@ 0000000180005038     libpopframe003.obj
 0002:00001060       ??_C@_03OFAPEBGM@?$CFs?6@  0000000180005060     libpopframe003.obj
 0002:00001068       ??_C@_0DM@LPIGEGNJ@s?2test?2hotspot?2jtreg?2vmTestbase@ 0000000180005068     libpopframe003.obj
 0002:000010a8       ??_C@_0CC@NFCNPEPK@Exception?5in?5JNI?5call?5?$CIcleared?$CJ@ 00000001800050a8     libpopframe003.obj
 0002:000010d0       ??_C@_0BJ@IBAKFIKF@jni?9?$DOExceptionDescribe?$CI?$CJ@ 00000001800050d0     libpopframe003.obj
 0002:000010f0       ??_C@_0BG@GGKALKMH@jni?9?$DOExceptionClear?$CI?$CJ@ 00000001800050f0     libpopframe003.obj
 0002:00001108       ??_C@_0CF@JMGFGJLJ@?$CD?5?5?5verified?5JNI?5assertion?5is?5F@ 0000000180005108     libpopframe003.obj
 0002:00001130       ??_C@_0CB@MLNJNCLJ@?5?5jvmti?5error?3?5code?$DN?$CFd?0?5name?$DN?$CFs@ 0000000180005130     libpopframe003.obj
 0002:00001158       ??_C@_0CD@OHBGDKMK@?$CD?5?5?5jvmti?5error?3?5code?$DN?$CFd?0?5name?$DN@ 0000000180005158     libpopframe003.obj
 0002:00001180       ??_C@_0CG@JNNCGPHB@?$CD?5?5?5error?5expected?3?5code?$DN?$CFd?0?5na@ 0000000180005180     libpopframe003.obj
 0002:000011b0       ??_C@_0EB@IMGKPCGE@?$CIstr_obj?5?$DN?5jni?9?$DONewStringUTF?$CIco@ 00000001800051b0     libpopframe003.obj
 0002:00001200       ??_C@_0EA@HFOGGBCC@s?2test?2hotspot?2jtreg?2vmTestbase@ 0000000180005200     libpopframe003.obj
 0002:00001240       ??_C@_0CB@PKFNCBLK@?$DO?$DO?$DO?$DO?$DO?$DO?$DO?$DO?5Invoke?5SuspendThread?$CI?$CJ@ 0000000180005240     libpopframe003.obj
 0002:00001268       ??_C@_0DC@FMKOEGFG@?$CFs?3?5Failed?5to?5call?5SuspendThrea@ 0000000180005268     libpopframe003.obj
 0002:000012a0       ??_C@_0CP@PCCFKDM@?$DM?$DM?$DM?$DM?$DM?$DM?$DM?$DM?5SuspendThread?$CI?$CJ?5is?5suc@ 00000001800052a0     libpopframe003.obj
 0002:000012d0       ??_C@_05KKCIMGE@error@     00000001800052d0     libpopframe003.obj
 0002:000012e0       ??_C@_0EA@PNBCDMOA@s?2test?2hotspot?2jtreg?2vmTestbase@ 00000001800052e0     libpopframe003.obj
 0002:00001320       ??_C@_0DI@ILAHDLMP@?$CI?$CKagentThreadProc?$CJ?$CIjvmti_env?0?5a@ 0000000180005320     libpopframe003.obj
 0002:00001358       ??_C@_0BD@KDBALNLB@JVMTI?5agent?5thread@ 0000000180005358     libpopframe003.obj
 0002:00001370       ??_C@_0BB@NOKBFPFO@java?1lang?1Thread@ 0000000180005370     libpopframe003.obj
 0002:00001384       ??_C@_06FALKBLGB@?$DMinit?$DO@ 0000000180005384     libpopframe003.obj
 0002:00001390       ??_C@_0BG@IKDDPPGD@?$CILjava?1lang?1String?$DL?$CJV@ 0000000180005390     libpopframe003.obj
 0002:000013b0       ??_C@_0EB@IFJBFEKC@?$CIthreadClass?5?$DN?5jni_env?9?$DOFindCla@ 00000001800053b0     libpopframe003.obj
 0002:00001400       ??_C@_0GF@FGFIBKKL@?$CIthreadCtor?5?$DN?5jni_env?9?$DOGetMetho@ 0000000180005400     libpopframe003.obj
 0002:00001468       ??_C@_0DN@NCPDJLOG@?$CIthreadName?5?$DN?5jni_env?9?$DONewStrin@ 0000000180005468     libpopframe003.obj
 0002:000014b0       ??_C@_0FE@PFKODBGC@?$CIthreadObject?5?$DN?5jni_env?9?$DONewObj@ 00000001800054b0     libpopframe003.obj
 0002:00001510       ??_C@_0ED@HOBAHHJI@?$CIthreadGlobalRef?5?$DN?5jni_env?9?$DONew@ 0000000180005510     libpopframe003.obj
 0002:00001560       ??_C@_0FN@HNJJAHFC@jvmti_env?9?$DORunAgentThread?$CIagent@ 0000000180005560     libpopframe003.obj
 0002:000015c0       ??_C@_0EA@MOJDNKDF@Debuggee?5status?5sync?5aborted?5be@ 00000001800055c0     libpopframe003.obj
 0002:00001600       ??_C@_0EA@EEOEJAEN@status?5?$DN?5syncDebuggeeStatus?$CIjni@ 0000000180005600     libpopframe003.obj
 0002:00001640       ??_C@_0BL@JBCFNBMB@nsk_jvmti_resetAgentData?$CI?$CJ@ 0000000180005640     libpopframe003.obj
 0002:00001660       ??_C@_0EL@LPBEELIP@s?2test?2hotspot?2jtreg?2vmTestbase@ 0000000180005660     libpopframe003.obj
 0002:000016b0       ??_C@_0CK@JDAMFDMJ@jvmti?9?$DOSetTag?$CIo?0?5tag?$CJ?5?$DN?$DN?5JVMTI_@ 00000001800056b0     libpopframe003.obj
 0002:000016e0       ??_C@_0CC@DAMNHKNI@Can?8t?5set?5tag?5?$CFli?5for?5object?5?$CFl@ 00000001800056e0     libpopframe003.obj
 0002:00001708       ??_C@_0DL@HAJPNKEF@jvmti?9?$DOGetObjectHashCode?$CIo?0?5?$CGha@ 0000000180005708     libpopframe003.obj
 0002:00001748       ??_C@_0BL@JFPIEOBF@Can?8t?5get?5hash?5object?5?$CFlx?6@ 0000000180005748     libpopframe003.obj
 0002:00001768       ??_C@_0BG@DICPHBKN@setTag?3?5?$CF08x?5?$DM?9?5?$CF?53li@ 0000000180005768     libpopframe003.obj
 0002:00001780       ??_C@_0DH@FCEEBDMJ@?$CIs?5?$DN?5jni?9?$DOGetStringUTFChars?$CIsIn@ 0000000180005780     libpopframe003.obj
 0002:000017b8       ??_C@_0BJ@OKKGHDCN@Can?8t?5get?5string?5at?5?$CF?$CDp?6@ 00000001800057b8     libpopframe003.obj
 0002:000017d8       ??_C@_0BP@EKFLGGFJ@Can?8t?5get?5string?5at?5?$CF?$CDp?3?5null?6@ 00000001800057d8     libpopframe003.obj
 0002:000017f8       ??_C@_06ICODBHCL@?5?1?1?5?$CFs@ 00000001800057f8     libpopframe003.obj
 0002:00001800       ??_C@_0DB@KGFPLEGO@?$CIr?5?$DN?5jvmti?9?$DOGetTag?$CIo?0?5?$CGtag?$CJ?$CJ?5?$DN?$DN@ 0000000180005800     libpopframe003.obj
 0002:00001838       ??_C@_0CO@PDAGBCGJ@Can?8t?5GetTag?5for?5object?5?$CFlx?4?5Re@ 0000000180005838     libpopframe003.obj
 0002:00001868       ??_C@_0CH@HPEODOHC@TEST_BUG?3?5Max?4?5number?5of?5refs?5r@ 0000000180005868     libpopframe003.obj
 0002:00001890       ??_C@_0DI@PHFCABIM@?$CIr?5?$DN?5jvmti?9?$DOGetTag?$CIfrom?0?5?$CGtagFr@ 0000000180005890     libpopframe003.obj
 0002:000018c8       ??_C@_0DI@MDEGFNKD@TEST_BUG?3?5Can?8t?5GetTag?5for?5obje@ 00000001800058c8     libpopframe003.obj
 0002:00001900       ??_C@_0DE@MLELJAHM@?$CIr?5?$DN?5jvmti?9?$DOGetTag?$CIto?0?5?$CGtagTo?$CJ?$CJ@ 0000000180005900     libpopframe003.obj
 0002:00001938       ??_C@_0CD@GAGNNEOH@?$CD?$CD?$CD?$CD?5FramePop?5event?5occurred?5?$CD?$CD@ 0000000180005938     libpopframe003.obj
 0002:00001960       ??_C@_0CF@CKNHIJHL@?$CD?$CD?$CD?$CD?5MethodExit?5event?5occurred?5@ 0000000180005960     libpopframe003.obj
 0002:00001990       ??_C@_0EP@PLDJJIHK@s?2test?2hotspot?2jtreg?2vmTestbase@ 0000000180005990     libpopframe003.obj
 0002:000019e0       ??_C@_0CA@LCONHFJP@?$DO?$DO?$DO?$DO?$DO?$DO?$DO?$DO?5Invoke?5ResumeThread?$CI?$CJ?6@ 00000001800059e0     libpopframe003.obj
 0002:00001a00       ??_C@_0DB@GNNPBNHM@?$CFs?3?5Failed?5to?5call?5ResumeThread@ 0000000180005a00     libpopframe003.obj
 0002:00001a38       ??_C@_0CO@ONBIKMHM@?$DM?$DM?$DM?$DM?$DM?$DM?$DM?$DM?5ResumeThread?$CI?$CJ?5is?5succ@ 0000000180005a38     libpopframe003.obj
 0002:00001a68       ??_C@_0CN@GHJIKGLO@Failed?5to?5enable?5METHOD_EXIT?5ev@ 0000000180005a68     libpopframe003.obj
 0002:00001a98       ??_C@_0CL@EPIEADBE@Failed?5to?5enable?5FRAME_POP?5even@ 0000000180005a98     libpopframe003.obj
 0002:00001ac8       ??_C@_0BM@MACMONCJ@?$DO?$DO?$DO?$DO?$DO?$DO?$DO?$DO?5Invoke?5PopFrame?$CI?$CJ?6@ 0000000180005ac8     libpopframe003.obj
 0002:00001af0       ??_C@_0EA@GKINCCCC@TEST?5FAILED?3?5the?5function?5PopFr@ 0000000180005af0     libpopframe003.obj
 0002:00001b30       ??_C@_0DF@KIBMOCOK@?7For?5more?5info?5about?5this?5error@ 0000000180005b30     libpopframe003.obj
 0002:00001b68       ??_C@_0DC@CHLBJIFK@Check?5?$CD1?5PASSED?3?5PopFrame?$CI?$CJ?5is?5@ 0000000180005b68     libpopframe003.obj
 0002:00001ba0       ??_C@_0EI@KHFEBDGK@TEST?5FAILED?3?5?$CFd?5JVMTI?5events?5we@ 0000000180005ba0     libpopframe003.obj
 0002:00001bf0       ??_C@_0EM@EAOIPNKK@Check?5?$CD2?5PASSED?3?5No?5JVMTI?5event@ 0000000180005bf0     libpopframe003.obj
 0002:00001c40       ??_C@_0CJ@KCDEKOCJ@Wrong?5result?5of?5a?5valid?5call?5to@ 0000000180005c40     libpopframe003.obj
 0002:00001c70       ??_C@_0DG@LAJPGIIE@?$CIGetPotentialCapabilities?$CJ?5unex@ 0000000180005c70     libpopframe003.obj
 0002:00001ca8       ??_C@_0CN@LKPEOJPO@?$CIAddCapabilities?$CJ?5unexpected?5er@ 0000000180005ca8     libpopframe003.obj
 0002:00001cd8       ??_C@_0CN@BCCBOHCH@?$CIGetCapabilities?$CJ?5unexpected?5er@ 0000000180005cd8     libpopframe003.obj
 0002:00001d08       ??_C@_0CG@MCCDAOGE@Warning?3?5PopFrame?5is?5not?5implem@ 0000000180005d08     libpopframe003.obj
 0002:00001d30       ??_C@_0CM@FEKJDMLD@Warning?3?5suspend?1resume?5is?5not?5@ 0000000180005d30     libpopframe003.obj
 0002:00001d60       ??_C@_0CP@IMINGNLL@?$CISetEventCallbacks?$CJ?5unexpected?5@ 0000000180005d60     libpopframe003.obj
 0002:00001d90       ??_C@_0DK@CDIPDFNJ@Warning?3?5FramePop?5or?5MethodExit@ 0000000180005d90     libpopframe003.obj
 0002:00001dd0       ??_C@_0BB@NOLAGKMP@watch_ev_monitor@ 0000000180005dd0     libpopframe003.obj
 0002:00001de8       ??_C@_0CO@BLGNGBDG@?$CICreateRawMonitor?$CJ?5unexpected?5e@ 0000000180005de8     libpopframe003.obj
 0002:00001e30       ??_C@_1EC@JIJBPKFM@?$AAa?$AAp?$AAi?$AA?9?$AAm?$AAs?$AA?9?$AAw?$AAi?$AAn?$AA?9?$AAc?$AAo?$AAr?$AAe@ 0000000180005e30     MSVCRT:thread_safe_statics.obj
 0002:00001e78       ??_C@_1BK@MGMFAEKH@?$AAk?$AAe?$AAr?$AAn?$AAe?$AAl?$AA3?$AA2?$AA?4?$AAd?$AAl?$AAl@ 0000000180005e78     MSVCRT:thread_safe_statics.obj
 0002:00001e98       ??_C@_0BJ@JEBJOJFJ@SleepConditionVariableCS@ 0000000180005e98     MSVCRT:thread_safe_statics.obj
 0002:00001eb8       ??_C@_0BJ@PGPPEPCC@WakeAllConditionVariable@ 0000000180005eb8     MSVCRT:thread_safe_statics.obj
 0002:00001ed8       _pDefaultRawDllMain        0000000180005ed8     MSVCRT:dll_dllmain.obj
 0002:00001ed8       _pRawDllMain               0000000180005ed8     MSVCRT:dll_dllmain.obj
 0002:00001ee0       __xmm@ffffffffffffffffffffffffffffffff 0000000180005ee0     MSVCRT:utility.obj
 0002:00001ef0       _load_config_used          0000000180005ef0     MSVCRT:loadcfg.obj
 0002:00002100       _tls_used                  0000000180006100     MSVCRT:tlssup.obj
 0002:00002128       __volatile_metadata        0000000180006128     <linker-defined>
 0002:000024f0       __rtc_iaa                  00000001800064f0     MSVCRT:initsect.obj
 0002:000024f8       __rtc_izz                  00000001800064f8     MSVCRT:initsect.obj
 0002:00002500       __rtc_taa                  0000000180006500     MSVCRT:initsect.obj
 0002:00002508       __rtc_tzz                  0000000180006508     MSVCRT:initsect.obj
 0002:00002510       _tls_start                 0000000180006510     MSVCRT:tlssup.obj
 0002:00002514       _Init_thread_epoch         0000000180006514     MSVCRT:thread_safe_statics.obj
 0002:00002518       _tls_end                   0000000180006518     MSVCRT:tlssup.obj
 0002:00002c00       __IMPORT_DESCRIPTOR_KERNEL32 0000000180006c00     kernel32:KERNEL32.dll
 0002:00002c14       __IMPORT_DESCRIPTOR_VCRUNTIME140 0000000180006c14     vcruntime:VCRUNTIME140.dll
 0002:00002c28       __IMPORT_DESCRIPTOR_api-ms-win-crt-runtime-l1-1-0 0000000180006c28     ucrt:api-ms-win-crt-runtime-l1-1-0.dll
 0002:00002c3c       __IMPORT_DESCRIPTOR_api-ms-win-crt-stdio-l1-1-0 0000000180006c3c     ucrt:api-ms-win-crt-stdio-l1-1-0.dll
 0002:00002c50       __IMPORT_DESCRIPTOR_api-ms-win-crt-string-l1-1-0 0000000180006c50     ucrt:api-ms-win-crt-string-l1-1-0.dll
 0002:00002c64       __NULL_IMPORT_DESCRIPTOR   0000000180006c64     kernel32:KERNEL32.dll
 0003:00000030       _Init_global_epoch         0000000180008030     MSVCRT:thread_safe_statics.obj
 0003:00000040       __security_cookie          0000000180008040     MSVCRT:gs_cookie.obj
 0003:00000048       __security_cookie_complement 0000000180008048     MSVCRT:gs_cookie.obj
 0003:00000050       __scrt_native_dllmain_reason 0000000180008050     MSVCRT:utility.obj
 0003:00000058       __isa_available            0000000180008058     MSVCRT:cpu_disp.obj
 0003:0000005c       __isa_enabled              000000018000805c     MSVCRT:cpu_disp.obj
 0003:00000060       __memset_fast_string_threshold 0000000180008060     MSVCRT:cpu_disp.obj
 0003:00000068       __memset_nt_threshold      0000000180008068     MSVCRT:cpu_disp.obj
 0003:00000070       __scrt_ucrt_dll_is_in_use  0000000180008070     MSVCRT:ucrt_stubs.obj
 0003:00000080       g_wrongHeapCallbacks       0000000180008080     libpopframe003.obj
 0003:00000100       g_szTagInfo                0000000180008100     libpopframe003.obj
 0003:00002040       g_tagFlags                 000000018000a040     libpopframe003.obj
 0003:00002428       g_refsToVerifyCnt          000000018000a428     libpopframe003.obj
 0003:0000242c       g_fakeUserData             000000018000a42c     libpopframe003.obj
 0003:00002430       g_tagVisitCount            000000018000a430     libpopframe003.obj
 0003:000033d0       g_refsToVerify             000000018000b3d0     libpopframe003.obj
 0003:0001aad0       g_userDataError            0000000180022ad0     libpopframe003.obj
 0003:0001adc8       ?_OptionsStorage@?1??__local_stdio_printf_options@@9@4_KA 0000000180022dc8     libpopframe003.obj
 0003:0001b388       _tls_index                 0000000180023388     MSVCRT:tlssup.obj
 0003:0001b390       __scrt_current_native_startup_state 0000000180023390     MSVCRT:utility.obj
 0003:0001b398       __scrt_native_startup_lock 0000000180023398     MSVCRT:utility.obj
 0003:0001b3d8       __scrt_debugger_hook_flag  00000001800233d8     MSVCRT:utility_desktop.obj
 0003:0001b3e0       ?__type_info_root_node@@3U__type_info_node@@A 00000001800233e0     MSVCRT:tncleanup.obj
 0003:0001b3f0       ?_OptionsStorage@?1??__local_stdio_scanf_options@@9@4_KA 00000001800233f0     MSVCRT:default_local_stdio_options.obj
 0003:0001b3f8       __favor                    00000001800233f8     MSVCRT:cpu_disp.obj
 0003:0001b400       __dyn_tls_init_callback    0000000180023400     <common>

 entry point at        0001:000024a0

 Static symbols

 0000:fffda000       .debug$S                   0000000180000000     popframe003.exp
 0000:fffda000       .debug$S                   0000000180000000     vcruntime:VCRUNTIME140.dll
 0000:fffda000       .debug$S                   0000000180000000     vcruntime:VCRUNTIME140.dll
 0000:fffda000       .debug$S                   0000000180000000     vcruntime:VCRUNTIME140.dll
 0000:fffda000       .debug$S                   0000000180000000     vcruntime:VCRUNTIME140.dll
 0000:fffda000       .debug$S                   0000000180000000     vcruntime:VCRUNTIME140.dll
 0000:fffda000       .debug$S                   0000000180000000     vcruntime:VCRUNTIME140.dll
 0000:fffda000       .debug$S                   0000000180000000     vcruntime:VCRUNTIME140.dll
 0000:fffda000       .debug$S                   0000000180000000     ucrt:api-ms-win-crt-convert-l1-1-0.dll
 0002:ffffc000       .idata$6                   0000000180000000     ucrt:api-ms-win-crt-convert-l1-1-0.dll
 0000:fffda000       .debug$S                   0000000180000000     ucrt:api-ms-win-crt-heap-l1-1-0.dll
 0000:fffda000       .debug$S                   0000000180000000     ucrt:api-ms-win-crt-heap-l1-1-0.dll
 0000:fffda000       .debug$S                   0000000180000000     ucrt:api-ms-win-crt-heap-l1-1-0.dll
 0000:fffda000       .debug$S                   0000000180000000     ucrt:api-ms-win-crt-heap-l1-1-0.dll
 0002:ffffc000       .idata$6                   0000000180000000     ucrt:api-ms-win-crt-heap-l1-1-0.dll
 0000:fffda000       .debug$S                   0000000180000000     ucrt:api-ms-win-crt-runtime-l1-1-0.dll
 0000:fffda000       .debug$S                   0000000180000000     ucrt:api-ms-win-crt-runtime-l1-1-0.dll
 0000:fffda000       .debug$S                   0000000180000000     ucrt:api-ms-win-crt-runtime-l1-1-0.dll
 0000:fffda000       .debug$S                   0000000180000000     ucrt:api-ms-win-crt-runtime-l1-1-0.dll
 0000:fffda000       .debug$S                   0000000180000000     ucrt:api-ms-win-crt-runtime-l1-1-0.dll
 0000:fffda000       .debug$S                   0000000180000000     ucrt:api-ms-win-crt-runtime-l1-1-0.dll
 0000:fffda000       .debug$S                   0000000180000000     ucrt:api-ms-win-crt-runtime-l1-1-0.dll
 0000:fffda000       .debug$S                   0000000180000000     ucrt:api-ms-win-crt-runtime-l1-1-0.dll
 0000:fffda000       .debug$S                   0000000180000000     ucrt:api-ms-win-crt-runtime-l1-1-0.dll
 0000:fffda000       .debug$S                   0000000180000000     ucrt:api-ms-win-crt-runtime-l1-1-0.dll
 0000:fffda000       .debug$S                   0000000180000000     ucrt:api-ms-win-crt-runtime-l1-1-0.dll
 0000:fffda000       .debug$S                   0000000180000000     ucrt:api-ms-win-crt-runtime-l1-1-0.dll
 0000:fffda000       .debug$S                   0000000180000000     ucrt:api-ms-win-crt-runtime-l1-1-0.dll
 0000:fffda000       .debug$S                   0000000180000000     ucrt:api-ms-win-crt-runtime-l1-1-0.dll
 0000:fffda000       .debug$S                   0000000180000000     ucrt:api-ms-win-crt-runtime-l1-1-0.dll
 0000:fffda000       .debug$S                   0000000180000000     ucrt:api-ms-win-crt-runtime-l1-1-0.dll
 0000:fffda000       .debug$S                   0000000180000000     ucrt:api-ms-win-crt-stdio-l1-1-0.dll
 0000:fffda000       .debug$S                   0000000180000000     ucrt:api-ms-win-crt-stdio-l1-1-0.dll
 0000:fffda000       .debug$S                   0000000180000000     ucrt:api-ms-win-crt-stdio-l1-1-0.dll
 0000:fffda000       .debug$S                   0000000180000000     ucrt:api-ms-win-crt-stdio-l1-1-0.dll
 0000:fffda000       .debug$S                   0000000180000000     ucrt:api-ms-win-crt-stdio-l1-1-0.dll
 0000:fffda000       .debug$S                   0000000180000000     ucrt:api-ms-win-crt-stdio-l1-1-0.dll
 0000:fffda000       .debug$S                   0000000180000000     ucrt:api-ms-win-crt-stdio-l1-1-0.dll
 0000:fffda000       .debug$S                   0000000180000000     ucrt:api-ms-win-crt-stdio-l1-1-0.dll
 0000:fffda000       .debug$S                   0000000180000000     ucrt:api-ms-win-crt-stdio-l1-1-0.dll
 0000:fffda000       .debug$S                   0000000180000000     ucrt:api-ms-win-crt-stdio-l1-1-0.dll
 0000:fffda000       .debug$S                   0000000180000000     ucrt:api-ms-win-crt-string-l1-1-0.dll
 0000:fffda000       .debug$S                   0000000180000000     ucrt:api-ms-win-crt-string-l1-1-0.dll
 0000:fffda000       .debug$S                   0000000180000000     ucrt:api-ms-win-crt-string-l1-1-0.dll
 0000:fffda000       .debug$S                   0000000180000000     ucrt:api-ms-win-crt-string-l1-1-0.dll
 0000:fffda000       .debug$S                   0000000180000000     ucrt:api-ms-win-crt-string-l1-1-0.dll
 0000:fffda000       .debug$S                   0000000180000000     ucrt:api-ms-win-crt-string-l1-1-0.dll
 0000:fffda000       .debug$S                   0000000180000000     ucrt:api-ms-win-crt-string-l1-1-0.dll
 0000:fffda000       .debug$S                   0000000180000000     ucrt:api-ms-win-crt-string-l1-1-0.dll
 0000:fffda000       .debug$S                   0000000180000000     kernel32:KERNEL32.dll
 0000:fffda000       .debug$S                   0000000180000000     kernel32:KERNEL32.dll
 0000:fffda000       .debug$S                   0000000180000000     kernel32:KERNEL32.dll
 0000:fffda000       .debug$S                   0000000180000000     kernel32:KERNEL32.dll
 0000:fffda000       .debug$S                   0000000180000000     kernel32:KERNEL32.dll
 0000:fffda000       .debug$S                   0000000180000000     kernel32:KERNEL32.dll
 0000:fffda000       .debug$S                   0000000180000000     kernel32:KERNEL32.dll
 0000:fffda000       .debug$S                   0000000180000000     kernel32:KERNEL32.dll
 0000:fffda000       .debug$S                   0000000180000000     kernel32:KERNEL32.dll
 0000:fffda000       .debug$S                   0000000180000000     kernel32:KERNEL32.dll
 0000:fffda000       .debug$S                   0000000180000000     kernel32:KERNEL32.dll
 0000:fffda000       .debug$S                   0000000180000000     kernel32:KERNEL32.dll
 0000:fffda000       .debug$S                   0000000180000000     kernel32:KERNEL32.dll
 0000:fffda000       .debug$S                   0000000180000000     kernel32:KERNEL32.dll
 0000:fffda000       .debug$S                   0000000180000000     kernel32:KERNEL32.dll
 0000:fffda000       .debug$S                   0000000180000000     kernel32:KERNEL32.dll
 0000:fffda000       .debug$S                   0000000180000000     kernel32:KERNEL32.dll
 0000:fffda000       .debug$S                   0000000180000000     kernel32:KERNEL32.dll
 0000:fffda000       .debug$S                   0000000180000000     kernel32:KERNEL32.dll
 0000:fffda000       .debug$S                   0000000180000000     kernel32:KERNEL32.dll
 0000:fffda000       .debug$S                   0000000180000000     kernel32:KERNEL32.dll
 0000:fffda000       .debug$S                   0000000180000000     kernel32:KERNEL32.dll
 0000:fffda000       .debug$S                   0000000180000000     kernel32:KERNEL32.dll
 0000:fffda000       .debug$S                   0000000180000000     kernel32:KERNEL32.dll
 0000:fffda000       .debug$S                   0000000180000000     kernel32:KERNEL32.dll
 0000:fffda000       .debug$S                   0000000180000000     kernel32:KERNEL32.dll
 0000:fffda000       .debug$S                   0000000180000000     kernel32:KERNEL32.dll
 0000:fffda000       .debug$S                   0000000180000000     kernel32:KERNEL32.dll
 0001:00001140       addRefToVerify             0000000180002140 f   libpopframe003.obj
 0001:000011b4       agentThreadWrapper         00000001800021b4 f   libpopframe003.obj
 0001:0000138c       file_basename              000000018000238c f   libpopframe003.obj
 0001:000019b4       startAgentThreadWrapper    00000001800029b4 f   libpopframe003.obj
 0001:00001ce0       syncDebuggeeStatus         0000000180002ce0 f   libpopframe003.obj
 0001:00001f68       capture_previous_context   0000000180002f68 f   MSVCRT:gs_report.obj
 0001:00001fdc       ?__scrt_initialize_thread_safe_statics@@YAHXZ 0000000180002fdc f   MSVCRT:thread_safe_statics.obj
 0001:000020ac       ?__scrt_uninitialize_thread_safe_statics@@YAXXZ 00000001800030ac f   MSVCRT:thread_safe_statics.obj
 0001:00002150       $$000000                   0000000180003150     MSVCRT:amdsecgs.obj
 0001:00002180       ?dllmain_crt_dispatch@@YAHQEAUHINSTANCE__@@KQEAX@Z 0000000180003180 f   MSVCRT:dll_dllmain.obj
 0001:000021d0       ?dllmain_crt_process_attach@@YAHQEAUHINSTANCE__@@QEAX@Z 00000001800031d0 f   MSVCRT:dll_dllmain.obj
 0001:000022e8       ?dllmain_crt_process_detach@@YAH_N@Z 00000001800032e8 f   MSVCRT:dll_dllmain.obj
 0001:0000236c       ?dllmain_dispatch@@YAHQEAUHINSTANCE__@@KQEAX@Z 000000018000336c f   MSVCRT:dll_dllmain.obj
 0001:00002d80       $$000000                   0000000180003d80     MSVCRT:guard_dispatch.obj
 0001:00002da0       $$000000                   0000000180003da0     MSVCRT:guard_xfg_dispatch.obj
 0001:00002db6       ?fin$0@?0??dllmain_crt_process_attach@@YAHQEAUHINSTANCE__@@QEAX@Z@4HA 0000000180003db6 f   MSVCRT:dll_dllmain.obj
 0001:00002dcd       ?fin$0@?0??dllmain_crt_process_detach@@YAH_N@Z@4HA 0000000180003dcd f   MSVCRT:dll_dllmain.obj
 0001:00002de6       ?fin$1@?0??dllmain_crt_process_detach@@YAH_N@Z@4HA 0000000180003de6 f   MSVCRT:dll_dllmain.obj
 0001:00002dfa       ?filt$0@?0??dllmain_dispatch@@YAHQEAUHINSTANCE__@@KQEAX@Z@4HA 0000000180003dfa f   MSVCRT:dll_dllmain.obj
 0001:00002e30       __scrt_is_nonwritable_in_current_image$filt$0 0000000180003e30 f   MSVCRT:utility.obj
 0002:000001e0       ?__scrt_initialize_tss_var@@3P6AHXZEA 00000001800041e0     MSVCRT:thread_safe_statics.obj
 0002:00000300       ?opcLengths@@3QBEB         0000000180004300     libpopframe003.obj
 0002:00001e18       GS_ExceptionPointers       0000000180005e18     MSVCRT:gs_report.obj
 0002:00002520       $unwind$fprintf            0000000180006520     libpopframe003.obj
 0002:0000252c       $unwind$printf             000000018000652c     libpopframe003.obj
 0002:00002538       $unwind$?NewObject@JNIEnv_@@QEAAPEAV_jobject@@PEAV_jclass@@PEAU_jmethodID@@ZZ 0000000180006538     libpopframe003.obj
 0002:00002538       $unwind$nsk_lcomplain      0000000180006538     libpopframe003.obj
 0002:00002538       $unwind$nsk_ldisplay       0000000180006538     libpopframe003.obj
 0002:00002540       $unwind$nsk_lvdisplay      0000000180006540     libpopframe003.obj
 0002:00002540       $unwind$_RTC_Initialize    0000000180006540     MSVCRT:initsect.obj
 0002:00002540       $unwind$_RTC_Terminate     0000000180006540     MSVCRT:initsect.obj
 0002:00002540       $unwind$?__scrt_initialize_thread_safe_statics@@YAHXZ 0000000180006540     MSVCRT:thread_safe_statics.obj
 0002:0000254c       $unwind$nsk_lvcomplain     000000018000654c     libpopframe003.obj
 0002:00002564       $unwind$nsk_ltrace         0000000180006564     libpopframe003.obj
 0002:00002564       $unwind$__report_gsfailure 0000000180006564     MSVCRT:gs_report.obj
 0002:0000256c       $unwind$Agent_Initialize   000000018000656c     libpopframe003.obj
 0002:0000256c       $unwind$Java_nsk_jvmti_PopFrame_popframe003_resThread 000000018000656c     libpopframe003.obj
 0002:0000256c       $unwind$Java_nsk_jvmti_PopFrame_popframe003_suspThread 000000018000656c     libpopframe003.obj
 0002:0000256c       $unwind$nsk_lvtrace        000000018000656c     libpopframe003.obj
 0002:0000256c       $unwind$__raise_securityfailure 000000018000656c     MSVCRT:gs_report.obj
 0002:0000256c       $unwind$__scrt_initialize_crt 000000018000656c     MSVCRT:utility.obj
 0002:0000256c       $unwind$__scrt_initialize_onexit_tables 000000018000656c     MSVCRT:utility.obj
 0002:0000256c       $unwind$__scrt_release_startup_lock 000000018000656c     MSVCRT:utility.obj
 0002:0000256c       $unwind$__scrt_uninitialize_crt 000000018000656c     MSVCRT:utility.obj
 0002:0000256c       $unwind$_onexit            000000018000656c     MSVCRT:utility.obj
 0002:00002574       $unwind$nsk_lverify        0000000180006574     libpopframe003.obj
 0002:00002584       $unwind$nsk_vprintf        0000000180006584     libpopframe003.obj
 0002:00002594       $unwind$nsk_printf         0000000180006594     libpopframe003.obj
 0002:0000259c       $unwind$?nsk_jni_lverify@@YAHHPEAUJNIEnv_@@HQEBDH1ZZ 000000018000659c     libpopframe003.obj
 0002:000025b0       $unwind$?nsk_jni_check_exception@@YAHPEAUJNIEnv_@@QEBDH@Z 00000001800065b0     libpopframe003.obj
 0002:000025cc       $unwind$FramePop           00000001800065cc     libpopframe003.obj
 0002:000025cc       $unwind$Java_nsk_jvmti_unit_FollowReferences_FollowRefObjects_resetTags 00000001800065cc     libpopframe003.obj
 0002:000025cc       $unwind$MethodExit         00000001800065cc     libpopframe003.obj
 0002:000025cc       $unwind$addRefToVerify     00000001800065cc     libpopframe003.obj
 0002:000025cc       $unwind$nsk_jvmti_resetAgentData 00000001800065cc     libpopframe003.obj
 0002:000025cc       $unwind$__scrt_initialize_default_local_stdio_options 00000001800065cc     MSVCRT:default_local_stdio_options.obj
 0002:000025cc       $unwind$?dllmain_crt_dispatch@@YAHQEAUHINSTANCE__@@KQEAX@Z 00000001800065cc     MSVCRT:dll_dllmain.obj
 0002:000025cc       $unwind$DllMain            00000001800065cc     MSVCRT:dll_dllmain_stub.obj
 0002:000025cc       $unwind$__GSHandlerCheck   00000001800065cc     MSVCRT:gshandler.obj
 0002:000025cc       $unwind$?__scrt_uninitialize_thread_safe_statics@@YAXXZ 00000001800065cc     MSVCRT:thread_safe_statics.obj
 0002:000025cc       $unwind$__scrt_acquire_startup_lock 00000001800065cc     MSVCRT:utility.obj
 0002:000025cc       $unwind$__scrt_dllmain_after_initialize_c 00000001800065cc     MSVCRT:utility.obj
 0002:000025cc       $unwind$__scrt_dllmain_before_initialize_c 00000001800065cc     MSVCRT:utility.obj
 0002:000025cc       $unwind$__scrt_dllmain_crt_thread_attach 00000001800065cc     MSVCRT:utility.obj
 0002:000025cc       $unwind$__scrt_dllmain_crt_thread_detach 00000001800065cc     MSVCRT:utility.obj
 0002:000025cc       $unwind$__scrt_dllmain_uninitialize_c 00000001800065cc     MSVCRT:utility.obj
 0002:000025cc       $unwind$__scrt_dllmain_uninitialize_critical 00000001800065cc     MSVCRT:utility.obj
 0002:000025cc       $unwind$atexit             00000001800065cc     MSVCRT:utility.obj
 0002:000025d4       $unwind$nsk_jvmti_lverify  00000001800065d4     libpopframe003.obj
 0002:000025e8       $unwind$exitOnError        00000001800065e8     libpopframe003.obj
 0002:000025f8       $unwind$Java_nsk_share_jvmti_ArgumentHandler_getAgentOptionsString 00000001800065f8     libpopframe003.obj
 0002:0000260c       $unwind$Java_nsk_jvmti_unit_FollowReferences_FollowRefObjects_getTag 000000018000660c     libpopframe003.obj
 0002:0000260c       $unwind$Java_nsk_share_jvmti_DebugeeClass_checkStatus 000000018000660c     libpopframe003.obj
 0002:0000260c       $unwind$agentThreadWrapper 000000018000660c     libpopframe003.obj
 0002:0000261c       $unwind$startAgentThreadWrapper 000000018000661c     libpopframe003.obj
 0002:00002638       $unwind$syncDebuggeeStatus 0000000180006638     libpopframe003.obj
 0002:00002638       $unwind$__scrt_dllmain_exception_filter 0000000180006638     MSVCRT:utility.obj
 0002:0000264c       $unwind$Java_nsk_share_jvmti_DebugeeClass_resetAgentData 000000018000664c     libpopframe003.obj
 0002:00002654       $unwind$MA_checkStatus     0000000180006654     libpopframe003.obj
 0002:00002668       $unwind$Java_nsk_jvmti_unit_FollowReferences_FollowRefObjects_setTag 0000000180006668     libpopframe003.obj
 0002:00002680       $unwind$Java_nsk_jvmti_unit_FollowReferences_FollowRefObjects_addRefToVerify 0000000180006680     libpopframe003.obj
 0002:0000269c       $unwind$Java_nsk_jvmti_PopFrame_popframe003_doPopFrame 000000018000669c     libpopframe003.obj
 0002:0000269c       $unwind$_DllMainCRTStartup 000000018000669c     MSVCRT:dll_dllmain.obj
 0002:000026ac       $unwind$capture_previous_context 00000001800066ac     MSVCRT:gs_report.obj
 0002:000026b8       $unwind$__GSHandlerCheckCommon 00000001800066b8     MSVCRT:gshandler.obj
 0002:000026c0       $xdatasym                  00000001800066c0     MSVCRT:amdsecgs.obj
 0002:000026c4       $unwind$?dllmain_crt_process_attach@@YAHQEAUHINSTANCE__@@QEAX@Z 00000001800066c4     MSVCRT:dll_dllmain.obj
 0002:00002700       $unwind$?fin$0@?0??dllmain_crt_process_attach@@YAHQEAUHINSTANCE__@@QEAX@Z@4HA 0000000180006700     MSVCRT:dll_dllmain.obj
 0002:00002700       $unwind$?fin$0@?0??dllmain_crt_process_detach@@YAH_N@Z@4HA 0000000180006700     MSVCRT:dll_dllmain.obj
 0002:00002700       $unwind$?fin$1@?0??dllmain_crt_process_detach@@YAH_N@Z@4HA 0000000180006700     MSVCRT:dll_dllmain.obj
 0002:00002708       $unwind$?dllmain_crt_process_detach@@YAH_N@Z 0000000180006708     MSVCRT:dll_dllmain.obj
 0002:0000275c       $unwind$?dllmain_dispatch@@YAHQEAUHINSTANCE__@@KQEAX@Z 000000018000675c     MSVCRT:dll_dllmain.obj
 0002:00002784       $unwind$?filt$0@?0??dllmain_dispatch@@YAHQEAUHINSTANCE__@@KQEAX@Z@4HA 0000000180006784     MSVCRT:dll_dllmain.obj
 0002:0000278c       $unwind$__scrt_is_nonwritable_in_current_image 000000018000678c     MSVCRT:utility.obj
 0002:000027ac       $unwind$__scrt_is_nonwritable_in_current_image$filt$0 00000001800067ac     MSVCRT:utility.obj
 0002:000027b4       $unwind$__scrt_fastfail    00000001800067b4     MSVCRT:utility_desktop.obj
 0002:000027c4       $unwind$__security_init_cookie 00000001800067c4     MSVCRT:gs_support.obj
 0002:000027d0       $unwind$__isa_available_init 00000001800067d0     MSVCRT:cpu_disp.obj
 0002:000027e0       $xdatasym                  00000001800067e0     MSVCRT:guard_dispatch.obj
 0002:000027e8       $xdatasym                  00000001800067e8     MSVCRT:guard_xfg_dispatch.obj
 0002:000027f0       .edata                     00000001800067f0     popframe003.exp
 0002:00002818       rgpv                       0000000180006818     popframe003.exp
 0002:0000285c       rgszName                   000000018000685c     popframe003.exp
 0002:000028a0       rgwOrd                     00000001800068a0     popframe003.exp
 0002:000028c2       szName                     00000001800068c2     popframe003.exp
 0002:000028d2       $N00001                    00000001800068d2     popframe003.exp
 0002:000028e1       $N00002                    00000001800068e1     popframe003.exp
 0002:000028ee       $N00003                    00000001800068ee     popframe003.exp
 0002:0000291d       $N00004                    000000018000691d     popframe003.exp
 0002:0000294b       $N00005                    000000018000694b     popframe003.exp
 0002:0000297a       $N00006                    000000018000697a     popframe003.exp
 0002:000029bf       $N00007                    00000001800069bf     popframe003.exp
 0002:000029fc       $N00008                    00000001800069fc     popframe003.exp
 0002:00002a44       $N00009                    0000000180006a44     popframe003.exp
 0002:00002a84       $N00010                    0000000180006a84     popframe003.exp
 0002:00002ac1       $N00011                    0000000180006ac1     popframe003.exp
 0002:00002afc       $N00012                    0000000180006afc     popframe003.exp
 0002:00002b2a       $N00013                    0000000180006b2a     popframe003.exp
 0002:00002b5b       $N00014                    0000000180006b5b     popframe003.exp
 0002:00002b8a       $N00015                    0000000180006b8a     popframe003.exp
 0002:00002bb9       $N00016                    0000000180006bb9     popframe003.exp
 0002:00002bee       $N00017                    0000000180006bee     popframe003.exp
 0002:00002ff2       .idata$6                   0000000180006ff2     kernel32:KERNEL32.dll
 0002:00003056       .idata$6                   0000000180007056     vcruntime:VCRUNTIME140.dll
 0002:000031b8       .idata$6                   00000001800071b8     ucrt:api-ms-win-crt-runtime-l1-1-0.dll
 0002:000031da       .idata$6                   00000001800071da     ucrt:api-ms-win-crt-stdio-l1-1-0.dll
 0002:000031fa       .idata$6                   00000001800071fa     ucrt:api-ms-win-crt-string-l1-1-0.dll
 0003:00000000       ?codeAttributeName@@3PEBDEB 0000000180008000     libpopframe003.obj
 0003:00000008       ?lineNumberAttributeName@@3PEBDEB 0000000180008008     libpopframe003.obj
 0003:00000010       ?localVarAttributeName@@3PEBDEB 0000000180008010     libpopframe003.obj
 0003:00000018       ?localVarTypeAttributeName@@3PEBDEB 0000000180008018     libpopframe003.obj
 0003:00000020       ?stackMapAttributeName@@3PEBDEB 0000000180008020     libpopframe003.obj
 0003:00000028       ?callBytes@@3PAEA          0000000180008028     libpopframe003.obj
 0003:0000002c       ?allocBytes@@3PAEA         000000018000802c     libpopframe003.obj
 0003:0001aad4       redefineAttempted          0000000180022ad4     libpopframe003.obj
 0003:0001aad8       nsk_context                0000000180022ad8     libpopframe003.obj
 0003:0001aae4       redefineSucceed            0000000180022ae4     libpopframe003.obj
 0003:0001aae8       agentFailed                0000000180022ae8     libpopframe003.obj
 0003:0001aaec       currentAgentStatus         0000000180022aec     libpopframe003.obj
 0003:0001aaf0       context                    0000000180022af0     libpopframe003.obj
 0003:0001aba8       agentThread                0000000180022ba8     libpopframe003.obj
 0003:0001abb0       agentThreadProc            0000000180022bb0     libpopframe003.obj
 0003:0001abb8       agentThreadArg             0000000180022bb8     libpopframe003.obj
 0003:0001abc0       agent_data                 0000000180022bc0     libpopframe003.obj
 0003:0001abd0       jvmti_env                  0000000180022bd0     libpopframe003.obj
 0003:0001abd8       jvm                        0000000180022bd8     libpopframe003.obj
 0003:0001abe0       jni_env                    0000000180022be0     libpopframe003.obj
 0003:0001abe8       checkStatus_func           0000000180022be8     libpopframe003.obj
 0003:0001abf0       ?codeAttributeIndex@@3GA   0000000180022bf0     libpopframe003.obj
 0003:0001abf4       ?lineNumberAttributeIndex@@3GA 0000000180022bf4     libpopframe003.obj
 0003:0001abf8       ?localVarAttributeIndex@@3GA 0000000180022bf8     libpopframe003.obj
 0003:0001abfc       ?localVarTypeAttributeIndex@@3GA 0000000180022bfc     libpopframe003.obj
 0003:0001ac00       ?stackMapAttributeIndex@@3GA 0000000180022c00     libpopframe003.obj
 0003:0001ac04       ?stackFrameOffset@@3GA     0000000180022c04     libpopframe003.obj
 0003:0001ac08       ?mode@@3HA                 0000000180022c08     libpopframe003.obj
 0003:0001ac0c       ?constantPoolSize@@3GA     0000000180022c0c     libpopframe003.obj
 0003:0001ac10       ?orig@@3PEBEEB             0000000180022c10     libpopframe003.obj
 0003:0001ac18       ?gen@@3PEAEEA              0000000180022c18     libpopframe003.obj
 0003:0001ac20       ?inputPos@@3PEAEEA         0000000180022c20     libpopframe003.obj
 0003:0001ac28       ?endPos@@3PEBEEB           0000000180022c28     libpopframe003.obj
 0003:0001ac30       ?genPos@@3PEAEEA           0000000180022c30     libpopframe003.obj
 0003:0001ac38       ?markPos@@3PEAEEA          0000000180022c38     libpopframe003.obj
 0003:0001ac40       ?constantPool@@3PEAPEADEA  0000000180022c40     libpopframe003.obj
 0003:0001ac48       ?constantPoolCount@@3GA    0000000180022c48     libpopframe003.obj
 0003:0001ac4c       ?zeroBytes@@3PAEA          0000000180022c4c     libpopframe003.obj
 0003:0001ac50       ?codeLength@@3IA           0000000180022c50     libpopframe003.obj
 0003:0001ac54       watch_ev                   0000000180022c54     libpopframe003.obj
 0003:0001ac58       ?map@@3PEAIEA              0000000180022c58     libpopframe003.obj
 0003:0001ac60       ?widening@@3PEACEA         0000000180022c60     libpopframe003.obj
 0003:0001ac68       jvmti                      0000000180022c68     libpopframe003.obj
 0003:0001ac70       caps                       0000000180022c70     libpopframe003.obj
 0003:0001ac80       callbacks                  0000000180022c80     libpopframe003.obj
 0003:0001adb8       gen_ev                     0000000180022db8     libpopframe003.obj
 0003:0001adbc       tot_result                 0000000180022dbc     libpopframe003.obj
 0003:0001adc0       watch_ev_monitor           0000000180022dc0     libpopframe003.obj
 0003:0001add0       GS_ExceptionRecord         0000000180022dd0     MSVCRT:gs_report.obj
 0003:0001ae70       GS_ContextRecord           0000000180022e70     MSVCRT:gs_report.obj
 0003:0001b340       ?g_tss_cv@@3U_RTL_CONDITION_VARIABLE@@A 0000000180023340     MSVCRT:thread_safe_statics.obj
 0003:0001b348       ?g_tss_event@@3PEAXEA      0000000180023348     MSVCRT:thread_safe_statics.obj
 0003:0001b350       ?g_tss_mutex@@3U_RTL_CRITICAL_SECTION@@A 0000000180023350     MSVCRT:thread_safe_statics.obj
 0003:0001b378       ?g_sleep_condition_variable_cs@@3P6AHPEAU_RTL_CONDITION_VARIABLE@@PEAU_RTL_CRITICAL_SECTION@@K@ZEA 0000000180023378     MSVCRT:thread_safe_statics.obj
 0003:0001b380       ?g_wake_all_condition_variable@@3P6AXPEAU_RTL_CONDITION_VARIABLE@@@ZEA 0000000180023380     MSVCRT:thread_safe_statics.obj
 0003:0001b38c       ?__proc_attached@@3HA      000000018002338c     MSVCRT:dll_dllmain.obj
 0003:0001b3a0       ?is_initialized_as_dll@@3_NA 00000001800233a0     MSVCRT:utility.obj
 0003:0001b3a1       ?module_local_atexit_table_initialized@@3_NA 00000001800233a1     MSVCRT:utility.obj
 0003:0001b3a8       ?module_local_atexit_table@@3U_onexit_table_t@@A 00000001800233a8     MSVCRT:utility.obj
 0003:0001b3c0       ?module_local_at_quick_exit_table@@3U_onexit_table_t@@A 00000001800233c0     MSVCRT:utility.obj
